 MethodBind

 Timestamp is 6fad8d27 (reproducible build file hash)

 Preferred load address is 0000000180000000

 Start         Length     Name                   Class
 0001:00000000 00003140H .text$mn                CODE
 0001:00003140 00000036H .text$mn$00             CODE
 0001:00003176 00000092H .text$x                 CODE
 0002:00000000 000001a0H .idata$5                DATA
 0002:000001a0 00000038H .00cfg                  DATA
 0002:000001d8 00000008H .CRT$XCA                DATA
 0002:000001e0 00000008H .CRT$XCZ                DATA
 0002:000001e8 00000008H .CRT$XIA                DATA
 0002:000001f0 00000008H .CRT$XIC                DATA
 0002:000001f8 00000008H .CRT$XIZ                DATA
 0002:00000200 00000008H .CRT$XLA                DATA
 0002:00000208 00000008H .CRT$XLZ                DATA
 0002:00000210 00000008H .CRT$XPA                DATA
 0002:00000218 00000008H .CRT$XPZ                DATA
 0002:00000220 00000008H .CRT$XTA                DATA
 0002:00000228 00000008H .CRT$XTZ                DATA
 0002:00000230 00000000H .gehcont$y              DATA
 0002:00000230 00000000H .gfids$y                DATA
 0002:00000230 00001e50H .rdata                  DATA
 0002:00002080 00000000H .rdata$CastGuardVftablesA DATA
 0002:00002080 00000000H .rdata$CastGuardVftablesC DATA
 0002:00002080 00000028H .rdata$T                DATA
 0002:000020a8 000000a4H .rdata$voltmd           DATA
 0002:0000214c 0000031cH .rdata$zzzdbg           DATA
 0002:00002468 00000008H .rtc$IAA                DATA
 0002:00002470 00000008H .rtc$IZZ                DATA
 0002:00002478 00000008H .rtc$TAA                DATA
 0002:00002480 00000008H .rtc$TZZ                DATA
 0002:00002488 00000004H .tls                    DATA
 0002:0000248c 00000004H .tls$                   DATA
 0002:00002490 00000008H .tls$ZZZ                DATA
 0002:00002498 00000318H .xdata                  DATA
 0002:000027b0 000005d0H .edata                  DATA
 0002:00002d80 00000064H .idata$2                DATA
 0002:00002de4 00000014H .idata$3                DATA
 0002:00002df8 000001a0H .idata$4                DATA
 0002:00002f98 00000428H .idata$6                DATA
 0003:00000000 00000080H .data                   DATA
 0003:00000080 0001f2a8H .bss                    DATA
 0004:00000000 00000408H .pdata                  DATA

  Address         Publics by Value              Rva+Base               Lib:Object

 0000:00000000       __AbsoluteZero             0000000000000000     <absolute>
 0000:00000000       ___safe_se_handler_count   0000000000000000     <absolute>
 0000:00000000       ___safe_se_handler_table   0000000000000000     <absolute>
 0000:00000000       __arm64x_extra_rfe_table   0000000000000000     <absolute>
 0000:00000000       __arm64x_extra_rfe_table_size 0000000000000000     <absolute>
 0000:00000000       __arm64x_native_entrypoint 0000000000000000     <absolute>
 0000:00000000       __arm64x_redirection_metadata 0000000000000000     <absolute>
 0000:00000000       __arm64x_redirection_metadata_count 0000000000000000     <absolute>
 0000:00000000       __dynamic_value_reloc_table 0000000000000000     <absolute>
 0000:00000000       __enclave_config           0000000000000000     <absolute>
 0000:00000000       __guard_check_icall_a64n_fptr 0000000000000000     <absolute>
 0000:00000000       __guard_eh_cont_count      0000000000000000     <absolute>
 0000:00000000       __guard_eh_cont_table      0000000000000000     <absolute>
 0000:00000000       __guard_fids_count         0000000000000000     <absolute>
 0000:00000000       __guard_fids_table         0000000000000000     <absolute>
 0000:00000000       __guard_iat_count          0000000000000000     <absolute>
 0000:00000000       __guard_iat_table          0000000000000000     <absolute>
 0000:00000000       __guard_longjmp_count      0000000000000000     <absolute>
 0000:00000000       __guard_longjmp_table      0000000000000000     <absolute>
 0000:00000000       __hybrid_auxiliary_iat     0000000000000000     <absolute>
 0000:00000000       __hybrid_auxiliary_iat_copy 0000000000000000     <absolute>
 0000:00000000       __hybrid_code_map          0000000000000000     <absolute>
 0000:00000000       __hybrid_code_map_count    0000000000000000     <absolute>
 0000:00000000       __x64_code_ranges_to_entry_points 0000000000000000     <absolute>
 0000:00000000       __x64_code_ranges_to_entry_points_count 0000000000000000     <absolute>
 0000:00000100       __guard_flags              0000000000000100     <absolute>
 0000:00000000       __ImageBase                0000000180000000     <linker-defined>
 0001:00000000       ?NewObject@JNIEnv_@@QEAAPEAV_jobject@@PEAV_jclass@@PEAU_jmethodID@@ZZ 0000000180001000 f i libMethodBind.obj
 0001:00000028       ?SetEventNotificationMode@_jvmtiEnv@@QEAA?AW4jvmtiError@@W4jvmtiEventMode@@W4jvmtiEvent@@PEAV_jobject@@ZZ 0000000180001028 f i libMethodBind.obj
 0001:00000034       ?TranslateError@@YAPEBDW4jvmtiError@@@Z 0000000180001034 f   libMethodBind.obj
 0001:000002ec       ?nsk_jni_check_exception@@YAHPEAUJNIEnv_@@QEBDH@Z 00000001800012ec f   libMethodBind.obj
 0001:00000430       ?nsk_jni_lverify@@YAHHPEAUJNIEnv_@@HQEBDH1ZZ 0000000180001430 f   libMethodBind.obj
 0001:000004d0       Agent_Initialize           00000001800014d0 f   libMethodBind.obj
 0001:00000678       Agent_OnAttach             0000000180001678 f   libMethodBind.obj
 0001:00000678       Agent_OnLoad               0000000180001678 f   libMethodBind.obj
 0001:00000680       Java_nsk_jvmti_unit_FollowReferences_FollowRefObjects_addRefToVerify 0000000180001680 f   libMethodBind.obj
 0001:00000858       Java_nsk_jvmti_unit_FollowReferences_FollowRefObjects_getTag 0000000180001858 f   libMethodBind.obj
 0001:00000918       Java_nsk_jvmti_unit_FollowReferences_FollowRefObjects_resetRefsToVerify 0000000180001918 f   libMethodBind.obj
 0001:00000920       Java_nsk_jvmti_unit_FollowReferences_FollowRefObjects_resetTags 0000000180001920 f   libMethodBind.obj
 0001:00000964       Java_nsk_jvmti_unit_FollowReferences_FollowRefObjects_setTag 0000000180001964 f   libMethodBind.obj
 0001:00000bbc       Java_nsk_jvmti_unit_MethodBind_JvmtiTest_CreateRawMonitor 0000000180001bbc f   libMethodBind.obj
 0001:00000c58       Java_nsk_jvmti_unit_MethodBind_JvmtiTest_GetFrameCount 0000000180001c58 f   libMethodBind.obj
 0001:00000cac       Java_nsk_jvmti_unit_MethodBind_JvmtiTest_GetResult 0000000180001cac f   libMethodBind.obj
 0001:00000cb4       Java_nsk_jvmti_unit_MethodBind_JvmtiTest_GetStackTrace 0000000180001cb4 f   libMethodBind.obj
 0001:00000d88       Java_nsk_jvmti_unit_MethodBind_JvmtiTest_RawMonitorEnter 0000000180001d88 f   libMethodBind.obj
 0001:00000de0       Java_nsk_jvmti_unit_MethodBind_JvmtiTest_RawMonitorExit 0000000180001de0 f   libMethodBind.obj
 0001:00000e38       Java_nsk_jvmti_unit_MethodBind_JvmtiTest_RawMonitorNotify 0000000180001e38 f   libMethodBind.obj
 0001:00000e90       Java_nsk_jvmti_unit_MethodBind_JvmtiTest_RawMonitorWait 0000000180001e90 f   libMethodBind.obj
 0001:00000eec       Java_nsk_jvmti_unit_MethodBind_JvmtiTest_SaveThreadInfo 0000000180001eec f   libMethodBind.obj
 0001:00000eec       _guard_check_icall_nop     0000000180001eec f   MSVCRT:guard_support.obj
 0001:00000ef0       Java_nsk_share_jvmti_ArgumentHandler_getAgentOptionsString 0000000180001ef0 f   libMethodBind.obj
 0001:00000fa0       Java_nsk_share_jvmti_DebugeeClass_checkStatus 0000000180001fa0 f   libMethodBind.obj
 0001:00001028       Java_nsk_share_jvmti_DebugeeClass_resetAgentData 0000000180002028 f   libMethodBind.obj
 0001:00001088       Java_nsk_share_jvmti_RedefineAgent_agentStatus 0000000180002088 f   libMethodBind.obj
 0001:00001094       Java_nsk_share_jvmti_RedefineAgent_isRedefined 0000000180002094 f   libMethodBind.obj
 0001:000010a0       Java_nsk_share_jvmti_RedefineAgent_redefineAttempted 00000001800020a0 f   libMethodBind.obj
 0001:000010ac       MA_checkStatus             00000001800020ac f   libMethodBind.obj
 0001:00001150       __local_stdio_printf_options 0000000180002150 f i libMethodBind.obj
 0001:00001158       _snprintf                  0000000180002158 f i libMethodBind.obj
 0001:00001388       debug_printf               0000000180002388 f   libMethodBind.obj
 0001:000013e4       exitOnError                00000001800023e4 f   libMethodBind.obj
 0001:00001498       fprintf                    0000000180002498 f i libMethodBind.obj
 0001:000014dc       init_callbacks             00000001800024dc f   libMethodBind.obj
 0001:00001524       my_findLoadedClass         0000000180002524 f   libMethodBind.obj
 0001:00001580       nsk_jvmti_lverify          0000000180002580 f   libMethodBind.obj
 0001:00001670       nsk_jvmti_resetAgentData   0000000180002670 f   libMethodBind.obj
 0001:000016f0       nsk_jvmti_setFailStatus    00000001800026f0 f   libMethodBind.obj
 0001:0000172c       nsk_lcomplain              000000018000272c f   libMethodBind.obj
 0001:0000174c       nsk_ldisplay               000000018000274c f   libMethodBind.obj
 0001:0000176c       nsk_ltrace                 000000018000276c f   libMethodBind.obj
 0001:0000178c       nsk_lvcomplain             000000018000278c f   libMethodBind.obj
 0001:00001944       nsk_lvdisplay              0000000180002944 f   libMethodBind.obj
 0001:00001990       nsk_lverify                0000000180002990 f   libMethodBind.obj
 0001:000019ec       nsk_lvtrace                00000001800029ec f   libMethodBind.obj
 0001:00001a4c       nsk_printf                 0000000180002a4c f   libMethodBind.obj
 0001:00001a74       nsk_vprintf                0000000180002a74 f   libMethodBind.obj
 0001:00001b28       print_method_name          0000000180002b28 f   libMethodBind.obj
 0001:00001bfc       printf                     0000000180002bfc f i libMethodBind.obj
 0001:00002124       testNativeMethodBind       0000000180003124 f   libMethodBind.obj
 0001:000021f8       vmExit                     00000001800031f8 f   libMethodBind.obj
 0001:00002204       vmInit                     0000000180003204 f   libMethodBind.obj
 0001:00002210       __raise_securityfailure    0000000180003210 f   MSVCRT:gs_report.obj
 0001:00002244       __report_gsfailure         0000000180003244 f   MSVCRT:gs_report.obj
 0001:00002484       __GSHandlerCheck           0000000180003484 f   MSVCRT:gshandler.obj
 0001:000024a4       __GSHandlerCheckCommon     00000001800034a4 f   MSVCRT:gshandler.obj
 0001:00002510       __security_check_cookie    0000000180003510 f   MSVCRT:amdsecgs.obj
 0001:00002850       _DllMainCRTStartup         0000000180003850 f   MSVCRT:dll_dllmain.obj
 0001:00002890       __scrt_acquire_startup_lock 0000000180003890 f   MSVCRT:utility.obj
 0001:000028cc       __scrt_dllmain_after_initialize_c 00000001800038cc f   MSVCRT:utility.obj
 0001:00002900       __scrt_dllmain_before_initialize_c 0000000180003900 f   MSVCRT:utility.obj
 0001:00002918       __scrt_dllmain_crt_thread_attach 0000000180003918 f   MSVCRT:utility.obj
 0001:00002940       __scrt_dllmain_crt_thread_detach 0000000180003940 f   MSVCRT:utility.obj
 0001:00002958       __scrt_dllmain_exception_filter 0000000180003958 f   MSVCRT:utility.obj
 0001:000029b8       __scrt_dllmain_uninitialize_c 00000001800039b8 f   MSVCRT:utility.obj
 0001:000029e8       __scrt_dllmain_uninitialize_critical 00000001800039e8 f   MSVCRT:utility.obj
 0001:000029fc       __scrt_initialize_crt      00000001800039fc f   MSVCRT:utility.obj
 0001:00002a48       __scrt_initialize_onexit_tables 0000000180003a48 f   MSVCRT:utility.obj
 0001:00002ad4       __scrt_is_nonwritable_in_current_image 0000000180003ad4 f   MSVCRT:utility.obj
 0001:00002b6c       __scrt_release_startup_lock 0000000180003b6c f   MSVCRT:utility.obj
 0001:00002b90       __scrt_uninitialize_crt    0000000180003b90 f   MSVCRT:utility.obj
 0001:00002bbc       _onexit                    0000000180003bbc f   MSVCRT:utility.obj
 0001:00002bf8       atexit                     0000000180003bf8 f   MSVCRT:utility.obj
 0001:00002c10       __crt_debugger_hook        0000000180003c10 f   MSVCRT:utility_desktop.obj
 0001:00002c18       __scrt_fastfail            0000000180003c18 f   MSVCRT:utility_desktop.obj
 0001:00002d64       __security_init_cookie     0000000180003d64 f   MSVCRT:gs_support.obj
 0001:00002e10       DllMain                    0000000180003e10 f   MSVCRT:dll_dllmain_stub.obj
 0001:00002e34       ?__scrt_initialize_type_info@@YAXXZ 0000000180003e34 f   MSVCRT:tncleanup.obj
 0001:00002e44       ?__scrt_uninitialize_type_info@@YAXXZ 0000000180003e44 f   MSVCRT:tncleanup.obj
 0001:00002e50       __local_stdio_scanf_options 0000000180003e50 f i MSVCRT:default_local_stdio_options.obj
 0001:00002e58       __scrt_initialize_default_local_stdio_options 0000000180003e58 f   MSVCRT:default_local_stdio_options.obj
 0001:00002e74       __scrt_get_dyn_tls_init_callback 0000000180003e74 f   MSVCRT:dyn_tls_init.obj
 0001:00002e7c       _RTC_Initialize            0000000180003e7c f   MSVCRT:initsect.obj
 0001:00002eb8       _RTC_Terminate             0000000180003eb8 f   MSVCRT:initsect.obj
 0001:00002ef4       __isa_available_init       0000000180003ef4 f   MSVCRT:cpu_disp.obj
 0001:000030a0       _get_startup_argv_mode     00000001800040a0 f   MSVCRT:argv_mode.obj
 0001:000030a8       __scrt_is_ucrt_dll_in_use  00000001800040a8 f   MSVCRT:ucrt_detection.obj
 0001:000030c0       memcpy                     00000001800040c0 f   vcruntime:VCRUNTIME140.dll
 0001:000030c6       memset                     00000001800040c6 f   vcruntime:VCRUNTIME140.dll
 0001:000030cc       strchr                     00000001800040cc f   vcruntime:VCRUNTIME140.dll
 0001:000030d2       strstr                     00000001800040d2 f   vcruntime:VCRUNTIME140.dll
 0001:000030d8       __C_specific_handler       00000001800040d8 f   vcruntime:VCRUNTIME140.dll
 0001:000030de       __std_type_info_destroy_list 00000001800040de f   vcruntime:VCRUNTIME140.dll
 0001:000030e4       strcmp                     00000001800040e4 f   ucrt:api-ms-win-crt-string-l1-1-0.dll
 0001:000030ea       strlen                     00000001800040ea f   ucrt:api-ms-win-crt-string-l1-1-0.dll
 0001:000030f0       _initterm                  00000001800040f0 f   ucrt:api-ms-win-crt-runtime-l1-1-0.dll
 0001:000030f6       _initterm_e                00000001800040f6 f   ucrt:api-ms-win-crt-runtime-l1-1-0.dll
 0001:000030fc       _seh_filter_dll            00000001800040fc f   ucrt:api-ms-win-crt-runtime-l1-1-0.dll
 0001:00003102       _configure_narrow_argv     0000000180004102 f   ucrt:api-ms-win-crt-runtime-l1-1-0.dll
 0001:00003108       _initialize_narrow_environment 0000000180004108 f   ucrt:api-ms-win-crt-runtime-l1-1-0.dll
 0001:0000310e       _initialize_onexit_table   000000018000410e f   ucrt:api-ms-win-crt-runtime-l1-1-0.dll
 0001:00003114       _register_onexit_function  0000000180004114 f   ucrt:api-ms-win-crt-runtime-l1-1-0.dll
 0001:0000311a       _execute_onexit_table      000000018000411a f   ucrt:api-ms-win-crt-runtime-l1-1-0.dll
 0001:00003120       _crt_atexit                0000000180004120 f   ucrt:api-ms-win-crt-runtime-l1-1-0.dll
 0001:00003126       _cexit                     0000000180004126 f   ucrt:api-ms-win-crt-runtime-l1-1-0.dll
 0001:0000312c       __acrt_initialize          000000018000412c f   MSVCRT:ucrt_stubs.obj
 0001:0000312c       __acrt_thread_attach       000000018000412c f   MSVCRT:ucrt_stubs.obj
 0001:0000312c       __acrt_thread_detach       000000018000412c f   MSVCRT:ucrt_stubs.obj
 0001:0000312c       __acrt_uninitialize        000000018000412c f   MSVCRT:ucrt_stubs.obj
 0001:0000312c       __acrt_uninitialize_critical 000000018000412c f   MSVCRT:ucrt_stubs.obj
 0001:0000312c       __scrt_stub_for_acrt_initialize 000000018000412c f   MSVCRT:ucrt_stubs.obj
 0001:0000312c       __scrt_stub_for_acrt_thread_attach 000000018000412c f   MSVCRT:ucrt_stubs.obj
 0001:0000312c       __scrt_stub_for_acrt_thread_detach 000000018000412c f   MSVCRT:ucrt_stubs.obj
 0001:0000312c       __scrt_stub_for_acrt_uninitialize 000000018000412c f   MSVCRT:ucrt_stubs.obj
 0001:0000312c       __scrt_stub_for_acrt_uninitialize_critical 000000018000412c f   MSVCRT:ucrt_stubs.obj
 0001:0000312c       __vcrt_initialize          000000018000412c f   MSVCRT:ucrt_stubs.obj
 0001:0000312c       __vcrt_thread_attach       000000018000412c f   MSVCRT:ucrt_stubs.obj
 0001:0000312c       __vcrt_thread_detach       000000018000412c f   MSVCRT:ucrt_stubs.obj
 0001:0000312c       __vcrt_uninitialize        000000018000412c f   MSVCRT:ucrt_stubs.obj
 0001:0000312c       __vcrt_uninitialize_critical 000000018000412c f   MSVCRT:ucrt_stubs.obj
 0001:00003130       __scrt_stub_for_is_c_termination_complete 0000000180004130 f   MSVCRT:ucrt_stubs.obj
 0001:00003130       _is_c_termination_complete 0000000180004130 f   MSVCRT:ucrt_stubs.obj
 0001:00003150       _guard_dispatch_icall_nop  0000000180004150 f   MSVCRT:guard_dispatch.obj
 0001:00003170       _guard_xfg_dispatch_icall_nop 0000000180004170 f   MSVCRT:guard_xfg_dispatch.obj
 0002:00000000       __imp_RtlCaptureContext    0000000180005000     kernel32:KERNEL32.dll
 0002:00000008       __imp_RtlLookupFunctionEntry 0000000180005008     kernel32:KERNEL32.dll
 0002:00000010       __imp_RtlVirtualUnwind     0000000180005010     kernel32:KERNEL32.dll
 0002:00000018       __imp_UnhandledExceptionFilter 0000000180005018     kernel32:KERNEL32.dll
 0002:00000020       __imp_SetUnhandledExceptionFilter 0000000180005020     kernel32:KERNEL32.dll
 0002:00000028       __imp_GetCurrentProcess    0000000180005028     kernel32:KERNEL32.dll
 0002:00000030       __imp_TerminateProcess     0000000180005030     kernel32:KERNEL32.dll
 0002:00000038       __imp_IsProcessorFeaturePresent 0000000180005038     kernel32:KERNEL32.dll
 0002:00000040       __imp_CloseHandle          0000000180005040     kernel32:KERNEL32.dll
 0002:00000048       __imp_InitializeCriticalSectionAndSpinCount 0000000180005048     kernel32:KERNEL32.dll
 0002:00000050       __imp_DeleteCriticalSection 0000000180005050     kernel32:KERNEL32.dll
 0002:00000058       __imp_CreateEventW         0000000180005058     kernel32:KERNEL32.dll
 0002:00000060       __imp_GetModuleHandleW     0000000180005060     kernel32:KERNEL32.dll
 0002:00000068       __imp_GetProcAddress       0000000180005068     kernel32:KERNEL32.dll
 0002:00000070       __imp_IsDebuggerPresent    0000000180005070     kernel32:KERNEL32.dll
 0002:00000078       __imp_QueryPerformanceCounter 0000000180005078     kernel32:KERNEL32.dll
 0002:00000080       __imp_GetCurrentProcessId  0000000180005080     kernel32:KERNEL32.dll
 0002:00000088       __imp_GetCurrentThreadId   0000000180005088     kernel32:KERNEL32.dll
 0002:00000090       __imp_GetSystemTimeAsFileTime 0000000180005090     kernel32:KERNEL32.dll
 0002:00000098       __imp_DisableThreadLibraryCalls 0000000180005098     kernel32:KERNEL32.dll
 0002:000000a0       __imp_InitializeSListHead  00000001800050a0     kernel32:KERNEL32.dll
 0002:000000a8       \177KERNEL32_NULL_THUNK_DATA 00000001800050a8     kernel32:KERNEL32.dll
 0002:000000b0       __imp_memcpy               00000001800050b0     vcruntime:VCRUNTIME140.dll
 0002:000000b8       __imp_memset               00000001800050b8     vcruntime:VCRUNTIME140.dll
 0002:000000c0       __imp_strchr               00000001800050c0     vcruntime:VCRUNTIME140.dll
 0002:000000c8       __imp_strstr               00000001800050c8     vcruntime:VCRUNTIME140.dll
 0002:000000d0       __imp___C_specific_handler 00000001800050d0     vcruntime:VCRUNTIME140.dll
 0002:000000d8       __imp___std_type_info_destroy_list 00000001800050d8     vcruntime:VCRUNTIME140.dll
 0002:000000e0       \177VCRUNTIME140_NULL_THUNK_DATA 00000001800050e0     vcruntime:VCRUNTIME140.dll
 0002:000000e8       __imp__errno               00000001800050e8     ucrt:api-ms-win-crt-runtime-l1-1-0.dll
 0002:000000f0       __imp_exit                 00000001800050f0     ucrt:api-ms-win-crt-runtime-l1-1-0.dll
 0002:000000f8       __imp__cexit               00000001800050f8     ucrt:api-ms-win-crt-runtime-l1-1-0.dll
 0002:00000100       __imp__crt_atexit          0000000180005100     ucrt:api-ms-win-crt-runtime-l1-1-0.dll
 0002:00000108       __imp__execute_onexit_table 0000000180005108     ucrt:api-ms-win-crt-runtime-l1-1-0.dll
 0002:00000110       __imp__register_onexit_function 0000000180005110     ucrt:api-ms-win-crt-runtime-l1-1-0.dll
 0002:00000118       __imp__initialize_onexit_table 0000000180005118     ucrt:api-ms-win-crt-runtime-l1-1-0.dll
 0002:00000120       __imp__initialize_narrow_environment 0000000180005120     ucrt:api-ms-win-crt-runtime-l1-1-0.dll
 0002:00000128       __imp__configure_narrow_argv 0000000180005128     ucrt:api-ms-win-crt-runtime-l1-1-0.dll
 0002:00000130       __imp__seh_filter_dll      0000000180005130     ucrt:api-ms-win-crt-runtime-l1-1-0.dll
 0002:00000138       __imp__initterm_e          0000000180005138     ucrt:api-ms-win-crt-runtime-l1-1-0.dll
 0002:00000140       __imp__initterm            0000000180005140     ucrt:api-ms-win-crt-runtime-l1-1-0.dll
 0002:00000148       \177api-ms-win-crt-runtime-l1-1-0_NULL_THUNK_DATA 0000000180005148     ucrt:api-ms-win-crt-runtime-l1-1-0.dll
 0002:00000150       __imp___acrt_iob_func      0000000180005150     ucrt:api-ms-win-crt-stdio-l1-1-0.dll
 0002:00000158       __imp_fflush               0000000180005158     ucrt:api-ms-win-crt-stdio-l1-1-0.dll
 0002:00000160       __imp___stdio_common_vsprintf 0000000180005160     ucrt:api-ms-win-crt-stdio-l1-1-0.dll
 0002:00000168       __imp___stdio_common_vfprintf 0000000180005168     ucrt:api-ms-win-crt-stdio-l1-1-0.dll
 0002:00000170       \177api-ms-win-crt-stdio-l1-1-0_NULL_THUNK_DATA 0000000180005170     ucrt:api-ms-win-crt-stdio-l1-1-0.dll
 0002:00000178       __imp_strcmp               0000000180005178     ucrt:api-ms-win-crt-string-l1-1-0.dll
 0002:00000180       __imp__strdup              0000000180005180     ucrt:api-ms-win-crt-string-l1-1-0.dll
 0002:00000180       __imp_strdup               0000000180005180     ucrt:api-ms-win-crt-string-l1-1-0.dll
 0002:00000188       __imp_strlen               0000000180005188     ucrt:api-ms-win-crt-string-l1-1-0.dll
 0002:00000190       __imp_strncpy              0000000180005190     ucrt:api-ms-win-crt-string-l1-1-0.dll
 0002:00000198       \177api-ms-win-crt-string-l1-1-0_NULL_THUNK_DATA 0000000180005198     ucrt:api-ms-win-crt-string-l1-1-0.dll
 0002:000001a0       __guard_check_icall_fptr   00000001800051a0     MSVCRT:guard_support.obj
 0002:000001a8       __guard_xfg_check_icall_fptr 00000001800051a8     MSVCRT:guard_support.obj
 0002:000001b0       __guard_dispatch_icall_fptr 00000001800051b0     MSVCRT:guard_support.obj
 0002:000001b8       __guard_xfg_dispatch_icall_fptr 00000001800051b8     MSVCRT:guard_support.obj
 0002:000001c0       __guard_xfg_table_dispatch_icall_fptr 00000001800051c0     MSVCRT:guard_support.obj
 0002:000001c8       __castguard_check_failure_os_handled_fptr 00000001800051c8     MSVCRT:guard_support.obj
 0002:000001d0       __guard_memcpy_fptr        00000001800051d0     vcruntime:softmemtag.obj
 0002:000001d8       __xc_a                     00000001800051d8     MSVCRT:initializers.obj
 0002:000001e0       __xc_z                     00000001800051e0     MSVCRT:initializers.obj
 0002:000001e8       __xi_a                     00000001800051e8     MSVCRT:initializers.obj
 0002:000001f8       __xi_z                     00000001800051f8     MSVCRT:initializers.obj
 0002:00000200       __xl_a                     0000000180005200     MSVCRT:tlssup.obj
 0002:00000208       __xl_z                     0000000180005208     MSVCRT:tlssup.obj
 0002:00000210       __xp_a                     0000000180005210     MSVCRT:initializers.obj
 0002:00000218       __xp_z                     0000000180005218     MSVCRT:initializers.obj
 0002:00000220       __xt_a                     0000000180005220     MSVCRT:initializers.obj
 0002:00000228       __xt_z                     0000000180005228     MSVCRT:initializers.obj
 0002:00000230       g_refKindStr               0000000180005230     libMethodBind.obj
 0002:000003e0       ??_C@_09BPLDFGCI@unknown_0@ 00000001800053e0     libMethodBind.obj
 0002:000003f0       ??_C@_0BL@FPNMECJD@JVMTI_HEAP_REFERENCE_CLASS@ 00000001800053f0     libMethodBind.obj
 0002:00000410       ??_C@_0BL@FKGKKLNM@JVMTI_HEAP_REFERENCE_FIELD@ 0000000180005410     libMethodBind.obj
 0002:00000430       ??_C@_0CD@CAEHCFJF@JVMTI_HEAP_REFERENCE_ARRAY_ELEM@ 0000000180005430     libMethodBind.obj
 0002:00000458       ??_C@_0CC@DNEBMCNK@JVMTI_HEAP_REFERENCE_CLASS_LOAD@ 0000000180005458     libMethodBind.obj
 0002:00000480       ??_C@_0BN@CJMIPEBB@JVMTI_HEAP_REFERENCE_SIGNERS@ 0000000180005480     libMethodBind.obj
 0002:000004a0       ??_C@_0CH@HBOIDPEB@JVMTI_HEAP_REFERENCE_PROTECTION@ 00000001800054a0     libMethodBind.obj
 0002:000004c8       ??_C@_0BP@MDKGDGKL@JVMTI_HEAP_REFERENCE_INTERFACE@ 00000001800054c8     libMethodBind.obj
 0002:000004e8       ??_C@_0CC@JJMIHNJH@JVMTI_HEAP_REFERENCE_STATIC_FIE@ 00000001800054e8     libMethodBind.obj
 0002:00000510       ??_C@_0CD@IDHEEGID@JVMTI_HEAP_REFERENCE_CONSTANT_P@ 0000000180005510     libMethodBind.obj
 0002:00000538       ??_C@_0CA@EFFCHNG@JVMTI_HEAP_REFERENCE_SUPERCLASS@ 0000000180005538     libMethodBind.obj
 0002:00000558       ??_C@_0L@PCDFHGCJ@unknown_11@ 0000000180005558     libMethodBind.obj
 0002:00000568       ??_C@_0L@NJBICFOK@unknown_12@ 0000000180005568     libMethodBind.obj
 0002:00000578       ??_C@_0L@MAADBEKL@unknown_13@ 0000000180005578     libMethodBind.obj
 0002:00000588       ??_C@_0L@IPECICGM@unknown_14@ 0000000180005588     libMethodBind.obj
 0002:00000598       ??_C@_0L@JGFJLDCN@unknown_15@ 0000000180005598     libMethodBind.obj
 0002:000005a8       ??_C@_0L@LNHEOAOO@unknown_16@ 00000001800055a8     libMethodBind.obj
 0002:000005b8       ??_C@_0L@KEGPNBKP@unknown_17@ 00000001800055b8     libMethodBind.obj
 0002:000005c8       ??_C@_0L@CDPHMNGA@unknown_18@ 00000001800055c8     libMethodBind.obj
 0002:000005d8       ??_C@_0L@DKOMPMCB@unknown_19@ 00000001800055d8     libMethodBind.obj
 0002:000005e8       ??_C@_0L@OJGIPJDB@unknown_20@ 00000001800055e8     libMethodBind.obj
 0002:000005f8       ??_C@_0CA@KAOFNDEM@JVMTI_HEAP_REFERENCE_JNI_GLOBAL@ 00000001800055f8     libMethodBind.obj
 0002:00000618       ??_C@_0CC@HPFAJBK@JVMTI_HEAP_REFERENCE_SYSTEM_CLA@ 0000000180005618     libMethodBind.obj
 0002:00000640       ??_C@_0BN@FDEGFOHC@JVMTI_HEAP_REFERENCE_MONITOR@ 0000000180005640     libMethodBind.obj
 0002:00000660       ??_C@_0CB@HKIBCMAJ@JVMTI_HEAP_REFERENCE_STACK_LOCA@ 0000000180005660     libMethodBind.obj
 0002:00000688       ??_C@_0BP@EAACMMOE@JVMTI_HEAP_REFERENCE_JNI_LOCAL@ 0000000180005688     libMethodBind.obj
 0002:000006a8       ??_C@_0BM@IJDEOGOE@JVMTI_HEAP_REFERENCE_THREAD@ 00000001800056a8     libMethodBind.obj
 0002:000006c8       ??_C@_0BL@EDGPPKC@JVMTI_HEAP_REFERENCE_OTHER@ 00000001800056c8     libMethodBind.obj
 0002:000006e4       ??_C@_04BCJPDBDA@Code@     00000001800056e4     libMethodBind.obj
 0002:000006f0       ??_C@_0BA@OCLMCFKC@LineNumberTable@ 00000001800056f0     libMethodBind.obj
 0002:00000700       ??_C@_0BD@CPAEPILC@LocalVariableTable@ 0000000180005700     libMethodBind.obj
 0002:00000718       ??_C@_0BH@NMBDNHBD@LocalVariableTypeTable@ 0000000180005718     libMethodBind.obj
 0002:00000730       ??_C@_0O@HIHEEDNJ@StackMapTable@ 0000000180005730     libMethodBind.obj
 0002:00000740       ??_C@_0L@HCDIAMJG@?9?5?$CFs?0?5?$CFd?3?5@ 0000000180005740     libMethodBind.obj
 0002:00000750       ??_C@_0JI@HLPECLFI@?$CD?5?4?4?4?6?$CD?5ERROR?3?5too?5many?5complai@ 0000000180005750     libMethodBind.obj
 0002:000007f0       ??_C@_0ED@JNEKCCOB@The?5following?5fake?5exception?5st@ 00000001800057f0     libMethodBind.obj
 0002:00000838       ??_C@_0CN@FCNMDFBH@nsk?4share?4Fake_Exception_for_RU@ 0000000180005838     libMethodBind.obj
 0002:00000868       ??_C@_08PGFFNAEI@?$CI?$CFs?3?$CFd?$CJ?5@ 0000000180005868     libMethodBind.obj
 0002:00000878       ??_C@_0DP@IENMAEGI@s?2test?2hotspot?2jtreg?2vmTestbase@ 0000000180005878     libMethodBind.obj
 0002:000008b8       ??_C@_0BL@NDJLFFJB@?7at?5nsk_lvcomplain?$CI?$CFs?3?$CFd?$CJ?6@ 00000001800058b8     libMethodBind.obj
 0002:000008d8       ??_C@_0BC@JOOKAFKF@?$CD?5ERROR?3?5?$CFs?0?5?$CFd?3?5@ 00000001800058d8     libMethodBind.obj
 0002:000008f0       ??_C@_09KJEAHMEH@?$CD?5ERROR?3?5@ 00000001800058f0     libMethodBind.obj
 0002:000008fc       ??_C@_02GPIOPFAK@?$DO?$DO@ 00000001800058fc     libMethodBind.obj
 0002:00000900       ??_C@_02FODMEDOG@?$DM?$DM@ 0000000180005900     libMethodBind.obj
 0002:00000904       ??_C@_02DJGKEECL@?4?4@     0000000180005904     libMethodBind.obj
 0002:00000908       ??_C@_0O@CJPGJOAF@?9?5?$CFs?0?5?$CFd?3?5?$CFs?5@ 0000000180005908     libMethodBind.obj
 0002:00000918       ??_C@_0CB@IAKPDOIC@?$CD?5?5?5verified?5assertion?5is?5FALSE@ 0000000180005918     libMethodBind.obj
 0002:00000940       ??_C@_0CO@LGONDEPD@stdout?3?5fflush?5failed?5?9?5err?$DN?$CFd?5@ 0000000180005940     libMethodBind.obj
 0002:00000970       ??_C@_0CO@KBGKJPBD@stderr?3?5fflush?5failed?5?9?5err?$DN?$CFd?5@ 0000000180005970     libMethodBind.obj
 0002:000009a0       ??_C@_0BB@JCNMKLLK@JVMTI_ERROR_NONE@ 00000001800059a0     libMethodBind.obj
 0002:000009b8       ??_C@_0BL@LDIMKLPH@JVMTI_ERROR_INVALID_THREAD@ 00000001800059b8     libMethodBind.obj
 0002:000009d8       ??_C@_0CB@PJFPAIKJ@JVMTI_ERROR_INVALID_THREAD_GROU@ 00000001800059d8     libMethodBind.obj
 0002:00000a00       ??_C@_0BN@LLMKHMNF@JVMTI_ERROR_INVALID_PRIORITY@ 0000000180005a00     libMethodBind.obj
 0002:00000a20       ??_C@_0CB@MBOFKAGB@JVMTI_ERROR_THREAD_NOT_SUSPENDE@ 0000000180005a20     libMethodBind.obj
 0002:00000a48       ??_C@_0BN@FABOLPBI@JVMTI_ERROR_THREAD_SUSPENDED@ 0000000180005a48     libMethodBind.obj
 0002:00000a68       ??_C@_0BN@FDGNOBJM@JVMTI_ERROR_THREAD_NOT_ALIVE@ 0000000180005a68     libMethodBind.obj
 0002:00000a88       ??_C@_0BL@GOBIFKNJ@JVMTI_ERROR_INVALID_OBJECT@ 0000000180005a88     libMethodBind.obj
 0002:00000aa8       ??_C@_0BK@FCMAJPPC@JVMTI_ERROR_INVALID_CLASS@ 0000000180005aa8     libMethodBind.obj
 0002:00000ac8       ??_C@_0BP@IKLLBKEB@JVMTI_ERROR_CLASS_NOT_PREPARED@ 0000000180005ac8     libMethodBind.obj
 0002:00000ae8       ??_C@_0BN@KLPPLKG@JVMTI_ERROR_INVALID_METHODID@ 0000000180005ae8     libMethodBind.obj
 0002:00000b08       ??_C@_0BN@BCEKOKND@JVMTI_ERROR_INVALID_LOCATION@ 0000000180005b08     libMethodBind.obj
 0002:00000b28       ??_C@_0BM@DFDGPME@JVMTI_ERROR_INVALID_FIELDID@ 0000000180005b28     libMethodBind.obj
 0002:00000b48       ??_C@_0BL@NELIEPEC@JVMTI_ERROR_NO_MORE_FRAMES@ 0000000180005b48     libMethodBind.obj
 0002:00000b68       ??_C@_0BJ@BDBECFDM@JVMTI_ERROR_OPAQUE_FRAME@ 0000000180005b68     libMethodBind.obj
 0002:00000b88       ??_C@_0BK@MIIFNLOB@JVMTI_ERROR_TYPE_MISMATCH@ 0000000180005b88     libMethodBind.obj
 0002:00000ba8       ??_C@_0BJ@HPCAOILC@JVMTI_ERROR_INVALID_SLOT@ 0000000180005ba8     libMethodBind.obj
 0002:00000bc8       ??_C@_0BG@CHILOPNI@JVMTI_ERROR_DUPLICATE@ 0000000180005bc8     libMethodBind.obj
 0002:00000be0       ??_C@_0BG@DIEMLHKM@JVMTI_ERROR_NOT_FOUND@ 0000000180005be0     libMethodBind.obj
 0002:00000bf8       ??_C@_0BM@NHMCKHOB@JVMTI_ERROR_INVALID_MONITOR@ 0000000180005bf8     libMethodBind.obj
 0002:00000c18       ??_C@_0BO@PPEDAJGL@JVMTI_ERROR_NOT_MONITOR_OWNER@ 0000000180005c18     libMethodBind.obj
 0002:00000c38       ??_C@_0BG@FCAIPEID@JVMTI_ERROR_INTERRUPT@ 0000000180005c38     libMethodBind.obj
 0002:00000c50       ??_C@_0CB@EGDBNKOI@JVMTI_ERROR_INVALID_CLASS_FORMA@ 0000000180005c50     libMethodBind.obj
 0002:00000c78       ??_C@_0CG@DGKOGIAL@JVMTI_ERROR_CIRCULAR_CLASS_DEFI@ 0000000180005c78     libMethodBind.obj
 0002:00000ca0       ??_C@_0BP@ICEALPKC@JVMTI_ERROR_FAILS_VERIFICATION@ 0000000180005ca0     libMethodBind.obj
 0002:00000cc0       ??_C@_0DC@JDACLMIO@JVMTI_ERROR_UNSUPPORTED_REDEFIN@ 0000000180005cc0     libMethodBind.obj
 0002:00000cf8       ??_C@_0DE@GKDKNOMJ@JVMTI_ERROR_UNSUPPORTED_REDEFIN@ 0000000180005cf8     libMethodBind.obj
 0002:00000d30       ??_C@_0BO@LAFKIOG@JVMTI_ERROR_INVALID_TYPESTATE@ 0000000180005d30     libMethodBind.obj
 0002:00000d50       ??_C@_0DH@INDGCLLB@JVMTI_ERROR_UNSUPPORTED_REDEFIN@ 0000000180005d50     libMethodBind.obj
 0002:00000d88       ??_C@_0DE@NHEOMMGI@JVMTI_ERROR_UNSUPPORTED_REDEFIN@ 0000000180005d88     libMethodBind.obj
 0002:00000dc0       ??_C@_0CA@EKPNJOEP@JVMTI_ERROR_UNSUPPORTED_VERSION@ 0000000180005dc0     libMethodBind.obj
 0002:00000de0       ??_C@_0BN@OFFMAHHL@JVMTI_ERROR_NAMES_DONT_MATCH@ 0000000180005de0     libMethodBind.obj
 0002:00000e00       ??_C@_0DN@HHBBLAKE@JVMTI_ERROR_UNSUPPORTED_REDEFIN@ 0000000180005e00     libMethodBind.obj
 0002:00000e40       ??_C@_0DO@HMBGBGNA@JVMTI_ERROR_UNSUPPORTED_REDEFIN@ 0000000180005e40     libMethodBind.obj
 0002:00000e80       ??_C@_0BP@PBECGKHJ@JVMTI_ERROR_UNMODIFIABLE_CLASS@ 0000000180005e80     libMethodBind.obj
 0002:00000ea0       ??_C@_0BK@CANILEHF@JVMTI_ERROR_NOT_AVAILABLE@ 0000000180005ea0     libMethodBind.obj
 0002:00000ec0       ??_C@_0CE@INJKMEFK@JVMTI_ERROR_MUST_POSSESS_CAPABI@ 0000000180005ec0     libMethodBind.obj
 0002:00000ee8       ??_C@_0BJ@LBFPFPDM@JVMTI_ERROR_NULL_POINTER@ 0000000180005ee8     libMethodBind.obj
 0002:00000f08       ??_C@_0BP@CHJPNNEM@JVMTI_ERROR_ABSENT_INFORMATION@ 0000000180005f08     libMethodBind.obj
 0002:00000f28       ??_C@_0BP@OMFMNLC@JVMTI_ERROR_INVALID_EVENT_TYPE@ 0000000180005f28     libMethodBind.obj
 0002:00000f48       ??_C@_0BN@BIBNPHHO@JVMTI_ERROR_ILLEGAL_ARGUMENT@ 0000000180005f48     libMethodBind.obj
 0002:00000f68       ??_C@_0BK@KKNDHDCE@JVMTI_ERROR_NATIVE_METHOD@ 0000000180005f68     libMethodBind.obj
 0002:00000f88       ??_C@_0BK@PMKCFHAE@JVMTI_ERROR_OUT_OF_MEMORY@ 0000000180005f88     libMethodBind.obj
 0002:00000fa8       ??_C@_0BK@NNJBDMNB@JVMTI_ERROR_ACCESS_DENIED@ 0000000180005fa8     libMethodBind.obj
 0002:00000fc8       ??_C@_0BI@GHECLMNC@JVMTI_ERROR_WRONG_PHASE@ 0000000180005fc8     libMethodBind.obj
 0002:00000fe0       ??_C@_0BF@OLIHJOII@JVMTI_ERROR_INTERNAL@ 0000000180005fe0     libMethodBind.obj
 0002:00000ff8       ??_C@_0BO@EOHGKJHI@JVMTI_ERROR_UNATTACHED_THREAD@ 0000000180005ff8     libMethodBind.obj
 0002:00001018       ??_C@_0CA@LKHFDACL@JVMTI_ERROR_INVALID_ENVIRONMENT@ 0000000180006018     libMethodBind.obj
 0002:00001038       ??_C@_0BA@MMFHLOKK@?$DMunknown?5error?$DO@ 0000000180006038     libMethodBind.obj
 0002:00001048       ??_C@_0CF@CBHOKDB@throwable?5?$DN?5jni?9?$DOExceptionOccur@ 0000000180006048     libMethodBind.obj
 0002:00001070       ??_C@_03OFAPEBGM@?$CFs?6@  0000000180006070     libMethodBind.obj
 0002:00001078       ??_C@_0DM@LPIGEGNJ@s?2test?2hotspot?2jtreg?2vmTestbase@ 0000000180006078     libMethodBind.obj
 0002:000010b8       ??_C@_0CC@NFCNPEPK@Exception?5in?5JNI?5call?5?$CIcleared?$CJ@ 00000001800060b8     libMethodBind.obj
 0002:000010e0       ??_C@_0BJ@IBAKFIKF@jni?9?$DOExceptionDescribe?$CI?$CJ@ 00000001800060e0     libMethodBind.obj
 0002:00001100       ??_C@_0BG@GGKALKMH@jni?9?$DOExceptionClear?$CI?$CJ@ 0000000180006100     libMethodBind.obj
 0002:00001118       ??_C@_0CF@JMGFGJLJ@?$CD?5?5?5verified?5JNI?5assertion?5is?5F@ 0000000180006118     libMethodBind.obj
 0002:00001140       ??_C@_0CB@MLNJNCLJ@?5?5jvmti?5error?3?5code?$DN?$CFd?0?5name?$DN?$CFs@ 0000000180006140     libMethodBind.obj
 0002:00001168       ??_C@_0CD@OHBGDKMK@?$CD?5?5?5jvmti?5error?3?5code?$DN?$CFd?0?5name?$DN@ 0000000180006168     libMethodBind.obj
 0002:00001190       ??_C@_0CG@JNNCGPHB@?$CD?5?5?5error?5expected?3?5code?$DN?$CFd?0?5na@ 0000000180006190     libMethodBind.obj
 0002:000011c0       ??_C@_0EB@IMGKPCGE@?$CIstr_obj?5?$DN?5jni?9?$DONewStringUTF?$CIco@ 00000001800061c0     libMethodBind.obj
 0002:00001210       ??_C@_0EA@HFOGGBCC@s?2test?2hotspot?2jtreg?2vmTestbase@ 0000000180006210     libMethodBind.obj
 0002:00001250       ??_C@_05KKCIMGE@error@     0000000180006250     libMethodBind.obj
 0002:00001258       ??_C@_0CJ@JACLEAA@Test?5failed?5by?5setFailStatus?$CI?$CJ?4@ 0000000180006258     libMethodBind.obj
 0002:00001290       ??_C@_0EA@PNBCDMOA@s?2test?2hotspot?2jtreg?2vmTestbase@ 0000000180006290     libMethodBind.obj
 0002:000012d0       ??_C@_0DI@ILAHDLMP@?$CI?$CKagentThreadProc?$CJ?$CIjvmti_env?0?5a@ 00000001800062d0     libMethodBind.obj
 0002:00001308       ??_C@_0BD@KDBALNLB@JVMTI?5agent?5thread@ 0000000180006308     libMethodBind.obj
 0002:00001320       ??_C@_0BB@NOKBFPFO@java?1lang?1Thread@ 0000000180006320     libMethodBind.obj
 0002:00001334       ??_C@_06FALKBLGB@?$DMinit?$DO@ 0000000180006334     libMethodBind.obj
 0002:00001340       ??_C@_0BG@IKDDPPGD@?$CILjava?1lang?1String?$DL?$CJV@ 0000000180006340     libMethodBind.obj
 0002:00001360       ??_C@_0EB@IFJBFEKC@?$CIthreadClass?5?$DN?5jni_env?9?$DOFindCla@ 0000000180006360     libMethodBind.obj
 0002:000013b0       ??_C@_0GF@FGFIBKKL@?$CIthreadCtor?5?$DN?5jni_env?9?$DOGetMetho@ 00000001800063b0     libMethodBind.obj
 0002:00001418       ??_C@_0DN@NCPDJLOG@?$CIthreadName?5?$DN?5jni_env?9?$DONewStrin@ 0000000180006418     libMethodBind.obj
 0002:00001460       ??_C@_0FE@PFKODBGC@?$CIthreadObject?5?$DN?5jni_env?9?$DONewObj@ 0000000180006460     libMethodBind.obj
 0002:000014c0       ??_C@_0ED@HOBAHHJI@?$CIthreadGlobalRef?5?$DN?5jni_env?9?$DONew@ 00000001800064c0     libMethodBind.obj
 0002:00001510       ??_C@_0FN@HNJJAHFC@jvmti_env?9?$DORunAgentThread?$CIagent@ 0000000180006510     libMethodBind.obj
 0002:00001570       ??_C@_0EA@MOJDNKDF@Debuggee?5status?5sync?5aborted?5be@ 0000000180006570     libMethodBind.obj
 0002:000015b0       ??_C@_0EA@EEOEJAEN@status?5?$DN?5syncDebuggeeStatus?$CIjni@ 00000001800065b0     libMethodBind.obj
 0002:000015f0       ??_C@_0BL@JBCFNBMB@nsk_jvmti_resetAgentData?$CI?$CJ@ 00000001800065f0     libMethodBind.obj
 0002:00001610       ??_C@_0EL@LPBEELIP@s?2test?2hotspot?2jtreg?2vmTestbase@ 0000000180006610     libMethodBind.obj
 0002:00001660       ??_C@_0CK@JDAMFDMJ@jvmti?9?$DOSetTag?$CIo?0?5tag?$CJ?5?$DN?$DN?5JVMTI_@ 0000000180006660     libMethodBind.obj
 0002:00001690       ??_C@_0CC@DAMNHKNI@Can?8t?5set?5tag?5?$CFli?5for?5object?5?$CFl@ 0000000180006690     libMethodBind.obj
 0002:000016b8       ??_C@_0DL@HAJPNKEF@jvmti?9?$DOGetObjectHashCode?$CIo?0?5?$CGha@ 00000001800066b8     libMethodBind.obj
 0002:000016f8       ??_C@_0BL@JFPIEOBF@Can?8t?5get?5hash?5object?5?$CFlx?6@ 00000001800066f8     libMethodBind.obj
 0002:00001718       ??_C@_0BG@DICPHBKN@setTag?3?5?$CF08x?5?$DM?9?5?$CF?53li@ 0000000180006718     libMethodBind.obj
 0002:00001730       ??_C@_0DH@FCEEBDMJ@?$CIs?5?$DN?5jni?9?$DOGetStringUTFChars?$CIsIn@ 0000000180006730     libMethodBind.obj
 0002:00001768       ??_C@_0BJ@OKKGHDCN@Can?8t?5get?5string?5at?5?$CF?$CDp?6@ 0000000180006768     libMethodBind.obj
 0002:00001788       ??_C@_0BP@EKFLGGFJ@Can?8t?5get?5string?5at?5?$CF?$CDp?3?5null?6@ 0000000180006788     libMethodBind.obj
 0002:000017a8       ??_C@_06ICODBHCL@?5?1?1?5?$CFs@ 00000001800067a8     libMethodBind.obj
 0002:000017b0       ??_C@_0DB@KGFPLEGO@?$CIr?5?$DN?5jvmti?9?$DOGetTag?$CIo?0?5?$CGtag?$CJ?$CJ?5?$DN?$DN@ 00000001800067b0     libMethodBind.obj
 0002:000017e8       ??_C@_0CO@PDAGBCGJ@Can?8t?5GetTag?5for?5object?5?$CFlx?4?5Re@ 00000001800067e8     libMethodBind.obj
 0002:00001818       ??_C@_0CH@HPEODOHC@TEST_BUG?3?5Max?4?5number?5of?5refs?5r@ 0000000180006818     libMethodBind.obj
 0002:00001840       ??_C@_0DI@PHFCABIM@?$CIr?5?$DN?5jvmti?9?$DOGetTag?$CIfrom?0?5?$CGtagFr@ 0000000180006840     libMethodBind.obj
 0002:00001878       ??_C@_0DI@MDEGFNKD@TEST_BUG?3?5Can?8t?5GetTag?5for?5obje@ 0000000180006878     libMethodBind.obj
 0002:000018b0       ??_C@_0DE@MLELJAHM@?$CIr?5?$DN?5jvmti?9?$DOGetTag?$CIto?0?5?$CGtagTo?$CJ?$CJ@ 00000001800068b0     libMethodBind.obj
 0002:000018e8       ??_C@_0O@PKEGMFDJ@VMInit?5event?6@ 00000001800068e8     libMethodBind.obj
 0002:000018f8       ??_C@_0P@OIDFFLDC@VMDeath?5event?6@ 00000001800068f8     libMethodBind.obj
 0002:00001908       ??_C@_0CI@JBBNPHEI@Intercepted?5findLoadedClass?0?5na@ 0000000180006908     libMethodBind.obj
 0002:00001930       ??_C@_0BE@LPEMBNKD@Error?3?5GetPhase?5?$CFd?6@ 0000000180006930     libMethodBind.obj
 0002:00001948       ??_C@_0O@GCHPOFEC@bind?5event?3?5?6@ 0000000180006948     libMethodBind.obj
 0002:00001958       ??_C@_0BA@OOPIAHLA@findLoadedClass@ 0000000180006958     libMethodBind.obj
 0002:00001968       ??_C@_0BM@NLMOBMHB@REDIRECTED?5findLoadedClass?6@ 0000000180006968     libMethodBind.obj
 0002:00001988       ??_C@_09OPJEJKBL@printdump@ 0000000180006988     libMethodBind.obj
 0002:00001998       ??_C@_0CJ@KCDEKOCJ@Wrong?5result?5of?5a?5valid?5call?5to@ 0000000180006998     libMethodBind.obj
 0002:000019c8       ??_C@_0CI@EDEMEGFA@GetPotentialCapabilities?5return@ 00000001800069c8     libMethodBind.obj
 0002:000019f0       ??_C@_03PMGGPEJJ@?$CFd?6@  00000001800069f0     libMethodBind.obj
 0002:000019f8       ??_C@_0BP@MCPPILG@AddCapabilities?5returned?5error@ 00000001800069f8     libMethodBind.obj
 0002:00001a18       ??_C@_0CB@NJBLABLF@SetEventCallbacks?5returned?5erro@ 0000000180006a18     libMethodBind.obj
 0002:00001a40       ??_C@_0DE@MEFKDHFM@SetEventNotificationMode?5for?5VM@ 0000000180006a40     libMethodBind.obj
 0002:00001a78       ??_C@_0DL@KHAEEJDH@SetEventNotificationMode?5for?5vm@ 0000000180006a78     libMethodBind.obj
 0002:00001ac0       ??_C@_0EF@JGCBFFDN@SetEventNotificationMode?5for?5na@ 0000000180006ac0     libMethodBind.obj
 0002:00001b08       ??_C@_0O@IEOHCAJP@Rawmonitor?9?$CFd@ 0000000180006b08     libMethodBind.obj
 0002:00001b18       ??_C@_0BL@PPNDBPKK@jvmti?5create?5raw?5monitor?5?6@ 0000000180006b18     libMethodBind.obj
 0002:00001b38       ??_C@_0CD@FAOAJHGL@Error?3?5ForceGarbageCollection?5?$CF@ 0000000180006b38     libMethodBind.obj
 0002:00001b60       ??_C@_0BK@KEFLCGDC@jvmti?5Raw?5monitor?5enter?5?6@ 0000000180006b60     libMethodBind.obj
 0002:00001b80       ??_C@_0BO@OJFPHDDP@Error?3?5Raw?5monitor?5enter?5?$CFd?5?6@ 0000000180006b80     libMethodBind.obj
 0002:00001ba0       ??_C@_0BJ@OJLKHENF@jvmti?5raw?5monitor?5exit?5?6@ 0000000180006ba0     libMethodBind.obj
 0002:00001bc0       ??_C@_0BL@GKGBEHOI@Error?3?5RawMonitorExit?5?$CFd?5?6@ 0000000180006bc0     libMethodBind.obj
 0002:00001be0       ??_C@_0BH@PILJFGHG@jvmti?5RawMonitorWait?5?6@ 0000000180006be0     libMethodBind.obj
 0002:00001bf8       ??_C@_0BL@EJFJOCBH@Error?3?5RawMonitorWait?5?$CFd?5?6@ 0000000180006bf8     libMethodBind.obj
 0002:00001c18       ??_C@_0BJ@DLFONEKK@jvmti?5RawMonitorNotify?5?6@ 0000000180006c18     libMethodBind.obj
 0002:00001c38       ??_C@_0BN@EJGKLMHH@Error?3?5RawMonitorNotify?5?$CFd?5?6@ 0000000180006c38     libMethodBind.obj
 0002:00001c58       ??_C@_0BG@MDNBHIDB@jvmti?5GetFrameCount?5?6@ 0000000180006c58     libMethodBind.obj
 0002:00001c70       ??_C@_0CE@CMHEGKH@Error?3?5GetFrameCount?5returned?5?5@ 0000000180006c70     libMethodBind.obj
 0002:00001c98       ??_C@_07CIFAGBMG@unknown@  0000000180006c98     libMethodBind.obj
 0002:00001ca0       ??_C@_0CF@HPJKBGDC@Error?3?5GetMethodDeclaringClass?5@ 0000000180006ca0     libMethodBind.obj
 0002:00001cc8       ??_C@_0BP@LFIKIAMN@Error?3?5GetClassSignature?5?$CFd?5?5?6@ 0000000180006cc8     libMethodBind.obj
 0002:00001ce8       ??_C@_0BL@OJMCGCKC@Error?3?5GetMethodName?5?$CFd?5?5?6@ 0000000180006ce8     libMethodBind.obj
 0002:00001d08       ??_C@_0M@JNIHOCAL@?$CFs?3?3?$CFs?$CI?$CFs?$CJ?6@ 0000000180006d08     libMethodBind.obj
 0002:00001d18       ??_C@_0CC@LBLLBNPM@Error?3?5Allocate?5failed?5with?5?5?$CFd@ 0000000180006d18     libMethodBind.obj
 0002:00001d40       ??_C@_0BK@FMLENDOH@Error?3?5GetStackTrace?5?$CFd?5?6@ 0000000180006d40     libMethodBind.obj
 0002:00001d60       ??_C@_0CE@LGABKEJM@Error?3?5Deallocate?5failed?5with?5?5@ 0000000180006d60     libMethodBind.obj
 0002:00001da0       ??_C@_1EC@JIJBPKFM@?$AAa?$AAp?$AAi?$AA?9?$AAm?$AAs?$AA?9?$AAw?$AAi?$AAn?$AA?9?$AAc?$AAo?$AAr?$AAe@ 0000000180006da0     MSVCRT:thread_safe_statics.obj
 0002:00001de8       ??_C@_1BK@MGMFAEKH@?$AAk?$AAe?$AAr?$AAn?$AAe?$AAl?$AA3?$AA2?$AA?4?$AAd?$AAl?$AAl@ 0000000180006de8     MSVCRT:thread_safe_statics.obj
 0002:00001e08       ??_C@_0BJ@JEBJOJFJ@SleepConditionVariableCS@ 0000000180006e08     MSVCRT:thread_safe_statics.obj
 0002:00001e28       ??_C@_0BJ@PGPPEPCC@WakeAllConditionVariable@ 0000000180006e28     MSVCRT:thread_safe_statics.obj
 0002:00001e48       _pDefaultRawDllMain        0000000180006e48     MSVCRT:dll_dllmain.obj
 0002:00001e48       _pRawDllMain               0000000180006e48     MSVCRT:dll_dllmain.obj
 0002:00001e50       __xmm@ffffffffffffffffffffffffffffffff 0000000180006e50     MSVCRT:utility.obj
 0002:00001e60       _load_config_used          0000000180006e60     MSVCRT:loadcfg.obj
 0002:00002080       _tls_used                  0000000180007080     MSVCRT:tlssup.obj
 0002:000020a8       __volatile_metadata        00000001800070a8     <linker-defined>
 0002:00002468       __rtc_iaa                  0000000180007468     MSVCRT:initsect.obj
 0002:00002470       __rtc_izz                  0000000180007470     MSVCRT:initsect.obj
 0002:00002478       __rtc_taa                  0000000180007478     MSVCRT:initsect.obj
 0002:00002480       __rtc_tzz                  0000000180007480     MSVCRT:initsect.obj
 0002:00002488       _tls_start                 0000000180007488     MSVCRT:tlssup.obj
 0002:0000248c       _Init_thread_epoch         000000018000748c     MSVCRT:thread_safe_statics.obj
 0002:00002490       _tls_end                   0000000180007490     MSVCRT:tlssup.obj
 0002:00002d80       __IMPORT_DESCRIPTOR_KERNEL32 0000000180007d80     kernel32:KERNEL32.dll
 0002:00002d94       __IMPORT_DESCRIPTOR_VCRUNTIME140 0000000180007d94     vcruntime:VCRUNTIME140.dll
 0002:00002da8       __IMPORT_DESCRIPTOR_api-ms-win-crt-runtime-l1-1-0 0000000180007da8     ucrt:api-ms-win-crt-runtime-l1-1-0.dll
 0002:00002dbc       __IMPORT_DESCRIPTOR_api-ms-win-crt-stdio-l1-1-0 0000000180007dbc     ucrt:api-ms-win-crt-stdio-l1-1-0.dll
 0002:00002dd0       __IMPORT_DESCRIPTOR_api-ms-win-crt-string-l1-1-0 0000000180007dd0     ucrt:api-ms-win-crt-string-l1-1-0.dll
 0002:00002de4       __NULL_IMPORT_DESCRIPTOR   0000000180007de4     kernel32:KERNEL32.dll
 0003:00000030       _Init_global_epoch         0000000180009030     MSVCRT:thread_safe_statics.obj
 0003:00000040       __security_cookie          0000000180009040     MSVCRT:gs_cookie.obj
 0003:00000048       __security_cookie_complement 0000000180009048     MSVCRT:gs_cookie.obj
 0003:00000050       __scrt_native_dllmain_reason 0000000180009050     MSVCRT:utility.obj
 0003:00000058       __isa_available            0000000180009058     MSVCRT:cpu_disp.obj
 0003:0000005c       __isa_enabled              000000018000905c     MSVCRT:cpu_disp.obj
 0003:00000060       __memset_fast_string_threshold 0000000180009060     MSVCRT:cpu_disp.obj
 0003:00000068       __memset_nt_threshold      0000000180009068     MSVCRT:cpu_disp.obj
 0003:00000070       __scrt_ucrt_dll_is_in_use  0000000180009070     MSVCRT:ucrt_stubs.obj
 0003:00000080       g_wrongHeapCallbacks       0000000180009080     libMethodBind.obj
 0003:00000100       g_szTagInfo                0000000180009100     libMethodBind.obj
 0003:00002040       g_tagFlags                 000000018000b040     libMethodBind.obj
 0003:00002428       g_refsToVerifyCnt          000000018000b428     libMethodBind.obj
 0003:0000242c       g_fakeUserData             000000018000b42c     libMethodBind.obj
 0003:00002430       g_tagVisitCount            000000018000b430     libMethodBind.obj
 0003:000033d0       g_refsToVerify             000000018000c3d0     libMethodBind.obj
 0003:0001aad0       g_userDataError            0000000180023ad0     libMethodBind.obj
 0003:0001aad4       iGlobalStatus              0000000180023ad4     libMethodBind.obj
 0003:0001aad8       jvmti                      0000000180023ad8     libMethodBind.obj
 0003:0001aae0       susp_thrd                  0000000180023ae0     libMethodBind.obj
 0003:0001e960       jraw_monitor               0000000180027960     libMethodBind.obj
 0003:0001ea00       process_once               0000000180027a00     libMethodBind.obj
 0003:0001ea04       printdump                  0000000180027a04     libMethodBind.obj
 0003:0001ea08       findLoadedClass_func       0000000180027a08     libMethodBind.obj
 0003:0001ece8       ?_OptionsStorage@?1??__local_stdio_printf_options@@9@4_KA 0000000180027ce8     libMethodBind.obj
 0003:0001f2a8       _tls_index                 00000001800282a8     MSVCRT:tlssup.obj
 0003:0001f2b0       __scrt_current_native_startup_state 00000001800282b0     MSVCRT:utility.obj
 0003:0001f2b8       __scrt_native_startup_lock 00000001800282b8     MSVCRT:utility.obj
 0003:0001f2f8       __scrt_debugger_hook_flag  00000001800282f8     MSVCRT:utility_desktop.obj
 0003:0001f300       ?__type_info_root_node@@3U__type_info_node@@A 0000000180028300     MSVCRT:tncleanup.obj
 0003:0001f310       ?_OptionsStorage@?1??__local_stdio_scanf_options@@9@4_KA 0000000180028310     MSVCRT:default_local_stdio_options.obj
 0003:0001f318       __favor                    0000000180028318     MSVCRT:cpu_disp.obj
 0003:0001f320       __dyn_tls_init_callback    0000000180028320     <common>

 entry point at        0001:00002850

 Static symbols

 0000:fffd5000       .debug$S                   0000000180000000     MethodBind.exp
 0000:fffd5000       .debug$S                   0000000180000000     vcruntime:VCRUNTIME140.dll
 0000:fffd5000       .debug$S                   0000000180000000     vcruntime:VCRUNTIME140.dll
 0000:fffd5000       .debug$S                   0000000180000000     vcruntime:VCRUNTIME140.dll
 0000:fffd5000       .debug$S                   0000000180000000     vcruntime:VCRUNTIME140.dll
 0000:fffd5000       .debug$S                   0000000180000000     vcruntime:VCRUNTIME140.dll
 0000:fffd5000       .debug$S                   0000000180000000     vcruntime:VCRUNTIME140.dll
 0000:fffd5000       .debug$S                   0000000180000000     vcruntime:VCRUNTIME140.dll
 0000:fffd5000       .debug$S                   0000000180000000     vcruntime:VCRUNTIME140.dll
 0000:fffd5000       .debug$S                   0000000180000000     ucrt:api-ms-win-crt-convert-l1-1-0.dll
 0002:ffffb000       .idata$6                   0000000180000000     ucrt:api-ms-win-crt-convert-l1-1-0.dll
 0000:fffd5000       .debug$S                   0000000180000000     ucrt:api-ms-win-crt-heap-l1-1-0.dll
 0000:fffd5000       .debug$S                   0000000180000000     ucrt:api-ms-win-crt-heap-l1-1-0.dll
 0000:fffd5000       .debug$S                   0000000180000000     ucrt:api-ms-win-crt-heap-l1-1-0.dll
 0000:fffd5000       .debug$S                   0000000180000000     ucrt:api-ms-win-crt-heap-l1-1-0.dll
 0002:ffffb000       .idata$6                   0000000180000000     ucrt:api-ms-win-crt-heap-l1-1-0.dll
 0000:fffd5000       .debug$S                   0000000180000000     ucrt:api-ms-win-crt-runtime-l1-1-0.dll
 0000:fffd5000       .debug$S                   0000000180000000     ucrt:api-ms-win-crt-runtime-l1-1-0.dll
 0000:fffd5000       .debug$S                   0000000180000000     ucrt:api-ms-win-crt-runtime-l1-1-0.dll
 0000:fffd5000       .debug$S                   0000000180000000     ucrt:api-ms-win-crt-runtime-l1-1-0.dll
 0000:fffd5000       .debug$S                   0000000180000000     ucrt:api-ms-win-crt-runtime-l1-1-0.dll
 0000:fffd5000       .debug$S                   0000000180000000     ucrt:api-ms-win-crt-runtime-l1-1-0.dll
 0000:fffd5000       .debug$S                   0000000180000000     ucrt:api-ms-win-crt-runtime-l1-1-0.dll
 0000:fffd5000       .debug$S                   0000000180000000     ucrt:api-ms-win-crt-runtime-l1-1-0.dll
 0000:fffd5000       .debug$S                   0000000180000000     ucrt:api-ms-win-crt-runtime-l1-1-0.dll
 0000:fffd5000       .debug$S                   0000000180000000     ucrt:api-ms-win-crt-runtime-l1-1-0.dll
 0000:fffd5000       .debug$S                   0000000180000000     ucrt:api-ms-win-crt-runtime-l1-1-0.dll
 0000:fffd5000       .debug$S                   0000000180000000     ucrt:api-ms-win-crt-runtime-l1-1-0.dll
 0000:fffd5000       .debug$S                   0000000180000000     ucrt:api-ms-win-crt-runtime-l1-1-0.dll
 0000:fffd5000       .debug$S                   0000000180000000     ucrt:api-ms-win-crt-runtime-l1-1-0.dll
 0000:fffd5000       .debug$S                   0000000180000000     ucrt:api-ms-win-crt-runtime-l1-1-0.dll
 0000:fffd5000       .debug$S                   0000000180000000     ucrt:api-ms-win-crt-runtime-l1-1-0.dll
 0000:fffd5000       .debug$S                   0000000180000000     ucrt:api-ms-win-crt-stdio-l1-1-0.dll
 0000:fffd5000       .debug$S                   0000000180000000     ucrt:api-ms-win-crt-stdio-l1-1-0.dll
 0000:fffd5000       .debug$S                   0000000180000000     ucrt:api-ms-win-crt-stdio-l1-1-0.dll
 0000:fffd5000       .debug$S                   0000000180000000     ucrt:api-ms-win-crt-stdio-l1-1-0.dll
 0000:fffd5000       .debug$S                   0000000180000000     ucrt:api-ms-win-crt-stdio-l1-1-0.dll
 0000:fffd5000       .debug$S                   0000000180000000     ucrt:api-ms-win-crt-stdio-l1-1-0.dll
 0000:fffd5000       .debug$S                   0000000180000000     ucrt:api-ms-win-crt-stdio-l1-1-0.dll
 0000:fffd5000       .debug$S                   0000000180000000     ucrt:api-ms-win-crt-stdio-l1-1-0.dll
 0000:fffd5000       .debug$S                   0000000180000000     ucrt:api-ms-win-crt-stdio-l1-1-0.dll
 0000:fffd5000       .debug$S                   0000000180000000     ucrt:api-ms-win-crt-stdio-l1-1-0.dll
 0000:fffd5000       .debug$S                   0000000180000000     ucrt:api-ms-win-crt-string-l1-1-0.dll
 0000:fffd5000       .debug$S                   0000000180000000     ucrt:api-ms-win-crt-string-l1-1-0.dll
 0000:fffd5000       .debug$S                   0000000180000000     ucrt:api-ms-win-crt-string-l1-1-0.dll
 0000:fffd5000       .debug$S                   0000000180000000     ucrt:api-ms-win-crt-string-l1-1-0.dll
 0000:fffd5000       .debug$S                   0000000180000000     ucrt:api-ms-win-crt-string-l1-1-0.dll
 0000:fffd5000       .debug$S                   0000000180000000     ucrt:api-ms-win-crt-string-l1-1-0.dll
 0000:fffd5000       .debug$S                   0000000180000000     ucrt:api-ms-win-crt-string-l1-1-0.dll
 0000:fffd5000       .debug$S                   0000000180000000     ucrt:api-ms-win-crt-string-l1-1-0.dll
 0000:fffd5000       .debug$S                   0000000180000000     kernel32:KERNEL32.dll
 0000:fffd5000       .debug$S                   0000000180000000     kernel32:KERNEL32.dll
 0000:fffd5000       .debug$S                   0000000180000000     kernel32:KERNEL32.dll
 0000:fffd5000       .debug$S                   0000000180000000     kernel32:KERNEL32.dll
 0000:fffd5000       .debug$S                   0000000180000000     kernel32:KERNEL32.dll
 0000:fffd5000       .debug$S                   0000000180000000     kernel32:KERNEL32.dll
 0000:fffd5000       .debug$S                   0000000180000000     kernel32:KERNEL32.dll
 0000:fffd5000       .debug$S                   0000000180000000     kernel32:KERNEL32.dll
 0000:fffd5000       .debug$S                   0000000180000000     kernel32:KERNEL32.dll
 0000:fffd5000       .debug$S                   0000000180000000     kernel32:KERNEL32.dll
 0000:fffd5000       .debug$S                   0000000180000000     kernel32:KERNEL32.dll
 0000:fffd5000       .debug$S                   0000000180000000     kernel32:KERNEL32.dll
 0000:fffd5000       .debug$S                   0000000180000000     kernel32:KERNEL32.dll
 0000:fffd5000       .debug$S                   0000000180000000     kernel32:KERNEL32.dll
 0000:fffd5000       .debug$S                   0000000180000000     kernel32:KERNEL32.dll
 0000:fffd5000       .debug$S                   0000000180000000     kernel32:KERNEL32.dll
 0000:fffd5000       .debug$S                   0000000180000000     kernel32:KERNEL32.dll
 0000:fffd5000       .debug$S                   0000000180000000     kernel32:KERNEL32.dll
 0000:fffd5000       .debug$S                   0000000180000000     kernel32:KERNEL32.dll
 0000:fffd5000       .debug$S                   0000000180000000     kernel32:KERNEL32.dll
 0000:fffd5000       .debug$S                   0000000180000000     kernel32:KERNEL32.dll
 0000:fffd5000       .debug$S                   0000000180000000     kernel32:KERNEL32.dll
 0000:fffd5000       .debug$S                   0000000180000000     kernel32:KERNEL32.dll
 0000:fffd5000       .debug$S                   0000000180000000     kernel32:KERNEL32.dll
 0000:fffd5000       .debug$S                   0000000180000000     kernel32:KERNEL32.dll
 0000:fffd5000       .debug$S                   0000000180000000     kernel32:KERNEL32.dll
 0000:fffd5000       .debug$S                   0000000180000000     kernel32:KERNEL32.dll
 0000:fffd5000       .debug$S                   0000000180000000     kernel32:KERNEL32.dll
 0001:000011b0       addRefToVerify             00000001800021b0 f   libMethodBind.obj
 0001:0000121c       agentThreadWrapper         000000018000221c f   libMethodBind.obj
 0001:00001468       file_basename              0000000180002468 f   libMethodBind.obj
 0001:00001c4c       startAgentThreadWrapper    0000000180002c4c f   libMethodBind.obj
 0001:00001f8c       syncDebuggeeStatus         0000000180002f8c f   libMethodBind.obj
 0001:00002318       capture_previous_context   0000000180003318 f   MSVCRT:gs_report.obj
 0001:0000238c       ?__scrt_initialize_thread_safe_statics@@YAHXZ 000000018000338c f   MSVCRT:thread_safe_statics.obj
 0001:0000245c       ?__scrt_uninitialize_thread_safe_statics@@YAXXZ 000000018000345c f   MSVCRT:thread_safe_statics.obj
 0001:00002500       $$000000                   0000000180003500     MSVCRT:amdsecgs.obj
 0001:00002530       ?dllmain_crt_dispatch@@YAHQEAUHINSTANCE__@@KQEAX@Z 0000000180003530 f   MSVCRT:dll_dllmain.obj
 0001:00002580       ?dllmain_crt_process_attach@@YAHQEAUHINSTANCE__@@QEAX@Z 0000000180003580 f   MSVCRT:dll_dllmain.obj
 0001:00002698       ?dllmain_crt_process_detach@@YAH_N@Z 0000000180003698 f   MSVCRT:dll_dllmain.obj
 0001:0000271c       ?dllmain_dispatch@@YAHQEAUHINSTANCE__@@KQEAX@Z 000000018000371c f   MSVCRT:dll_dllmain.obj
 0001:00003140       $$000000                   0000000180004140     MSVCRT:guard_dispatch.obj
 0001:00003160       $$000000                   0000000180004160     MSVCRT:guard_xfg_dispatch.obj
 0001:00003176       ?fin$0@?0??dllmain_crt_process_attach@@YAHQEAUHINSTANCE__@@QEAX@Z@4HA 0000000180004176 f   MSVCRT:dll_dllmain.obj
 0001:0000318d       ?fin$0@?0??dllmain_crt_process_detach@@YAH_N@Z@4HA 000000018000418d f   MSVCRT:dll_dllmain.obj
 0001:000031a6       ?fin$1@?0??dllmain_crt_process_detach@@YAH_N@Z@4HA 00000001800041a6 f   MSVCRT:dll_dllmain.obj
 0001:000031ba       ?filt$0@?0??dllmain_dispatch@@YAHQEAUHINSTANCE__@@KQEAX@Z@4HA 00000001800041ba f   MSVCRT:dll_dllmain.obj
 0001:000031f0       __scrt_is_nonwritable_in_current_image$filt$0 00000001800041f0 f   MSVCRT:utility.obj
 0002:000001f0       ?__scrt_initialize_tss_var@@3P6AHXZEA 00000001800051f0     MSVCRT:thread_safe_statics.obj
 0002:00000310       ?opcLengths@@3QBEB         0000000180005310     libMethodBind.obj
 0002:00001d88       GS_ExceptionPointers       0000000180006d88     MSVCRT:gs_report.obj
 0002:00002498       $unwind$fprintf            0000000180007498     libMethodBind.obj
 0002:000024a4       $unwind$printf             00000001800074a4     libMethodBind.obj
 0002:000024b0       $unwind$_snprintf          00000001800074b0     libMethodBind.obj
 0002:000024c0       $unwind$?NewObject@JNIEnv_@@QEAAPEAV_jobject@@PEAV_jclass@@PEAU_jmethodID@@ZZ 00000001800074c0     libMethodBind.obj
 0002:000024c0       $unwind$nsk_lcomplain      00000001800074c0     libMethodBind.obj
 0002:000024c0       $unwind$nsk_ldisplay       00000001800074c0     libMethodBind.obj
 0002:000024c8       $unwind$nsk_lvdisplay      00000001800074c8     libMethodBind.obj
 0002:000024c8       $unwind$_RTC_Initialize    00000001800074c8     MSVCRT:initsect.obj
 0002:000024c8       $unwind$_RTC_Terminate     00000001800074c8     MSVCRT:initsect.obj
 0002:000024c8       $unwind$?__scrt_initialize_thread_safe_statics@@YAHXZ 00000001800074c8     MSVCRT:thread_safe_statics.obj
 0002:000024d4       $unwind$nsk_lvcomplain     00000001800074d4     libMethodBind.obj
 0002:000024ec       $unwind$nsk_ltrace         00000001800074ec     libMethodBind.obj
 0002:000024ec       $unwind$__report_gsfailure 00000001800074ec     MSVCRT:gs_report.obj
 0002:000024f4       $unwind$Java_nsk_jvmti_unit_MethodBind_JvmtiTest_GetFrameCount 00000001800074f4     libMethodBind.obj
 0002:000024f4       $unwind$Java_nsk_jvmti_unit_MethodBind_JvmtiTest_RawMonitorEnter 00000001800074f4     libMethodBind.obj
 0002:000024f4       $unwind$Java_nsk_jvmti_unit_MethodBind_JvmtiTest_RawMonitorExit 00000001800074f4     libMethodBind.obj
 0002:000024f4       $unwind$Java_nsk_jvmti_unit_MethodBind_JvmtiTest_RawMonitorNotify 00000001800074f4     libMethodBind.obj
 0002:000024f4       $unwind$Java_nsk_jvmti_unit_MethodBind_JvmtiTest_RawMonitorWait 00000001800074f4     libMethodBind.obj
 0002:000024f4       $unwind$nsk_lvtrace        00000001800074f4     libMethodBind.obj
 0002:000024f4       $unwind$__raise_securityfailure 00000001800074f4     MSVCRT:gs_report.obj
 0002:000024f4       $unwind$__scrt_initialize_crt 00000001800074f4     MSVCRT:utility.obj
 0002:000024f4       $unwind$__scrt_initialize_onexit_tables 00000001800074f4     MSVCRT:utility.obj
 0002:000024f4       $unwind$__scrt_release_startup_lock 00000001800074f4     MSVCRT:utility.obj
 0002:000024f4       $unwind$__scrt_uninitialize_crt 00000001800074f4     MSVCRT:utility.obj
 0002:000024f4       $unwind$_onexit            00000001800074f4     MSVCRT:utility.obj
 0002:000024fc       $unwind$nsk_lverify        00000001800074fc     libMethodBind.obj
 0002:0000250c       $unwind$nsk_vprintf        000000018000750c     libMethodBind.obj
 0002:0000251c       $unwind$nsk_printf         000000018000751c     libMethodBind.obj
 0002:00002524       $unwind$?nsk_jni_lverify@@YAHHPEAUJNIEnv_@@HQEBDH1ZZ 0000000180007524     libMethodBind.obj
 0002:00002538       $unwind$?nsk_jni_check_exception@@YAHPEAUJNIEnv_@@QEBDH@Z 0000000180007538     libMethodBind.obj
 0002:00002554       $unwind$Java_nsk_jvmti_unit_FollowReferences_FollowRefObjects_resetTags 0000000180007554     libMethodBind.obj
 0002:00002554       $unwind$addRefToVerify     0000000180007554     libMethodBind.obj
 0002:00002554       $unwind$init_callbacks     0000000180007554     libMethodBind.obj
 0002:00002554       $unwind$nsk_jvmti_resetAgentData 0000000180007554     libMethodBind.obj
 0002:00002554       $unwind$nsk_jvmti_setFailStatus 0000000180007554     libMethodBind.obj
 0002:00002554       $unwind$__scrt_initialize_default_local_stdio_options 0000000180007554     MSVCRT:default_local_stdio_options.obj
 0002:00002554       $unwind$?dllmain_crt_dispatch@@YAHQEAUHINSTANCE__@@KQEAX@Z 0000000180007554     MSVCRT:dll_dllmain.obj
 0002:00002554       $unwind$DllMain            0000000180007554     MSVCRT:dll_dllmain_stub.obj
 0002:00002554       $unwind$__GSHandlerCheck   0000000180007554     MSVCRT:gshandler.obj
 0002:00002554       $unwind$?__scrt_uninitialize_thread_safe_statics@@YAXXZ 0000000180007554     MSVCRT:thread_safe_statics.obj
 0002:00002554       $unwind$__scrt_acquire_startup_lock 0000000180007554     MSVCRT:utility.obj
 0002:00002554       $unwind$__scrt_dllmain_after_initialize_c 0000000180007554     MSVCRT:utility.obj
 0002:00002554       $unwind$__scrt_dllmain_before_initialize_c 0000000180007554     MSVCRT:utility.obj
 0002:00002554       $unwind$__scrt_dllmain_crt_thread_attach 0000000180007554     MSVCRT:utility.obj
 0002:00002554       $unwind$__scrt_dllmain_crt_thread_detach 0000000180007554     MSVCRT:utility.obj
 0002:00002554       $unwind$__scrt_dllmain_uninitialize_c 0000000180007554     MSVCRT:utility.obj
 0002:00002554       $unwind$__scrt_dllmain_uninitialize_critical 0000000180007554     MSVCRT:utility.obj
 0002:00002554       $unwind$atexit             0000000180007554     MSVCRT:utility.obj
 0002:0000255c       $unwind$nsk_jvmti_lverify  000000018000755c     libMethodBind.obj
 0002:00002570       $unwind$exitOnError        0000000180007570     libMethodBind.obj
 0002:00002580       $unwind$Java_nsk_share_jvmti_ArgumentHandler_getAgentOptionsString 0000000180007580     libMethodBind.obj
 0002:00002594       $unwind$Java_nsk_jvmti_unit_FollowReferences_FollowRefObjects_getTag 0000000180007594     libMethodBind.obj
 0002:00002594       $unwind$Java_nsk_share_jvmti_DebugeeClass_checkStatus 0000000180007594     libMethodBind.obj
 0002:00002594       $unwind$agentThreadWrapper 0000000180007594     libMethodBind.obj
 0002:000025a4       $unwind$startAgentThreadWrapper 00000001800075a4     libMethodBind.obj
 0002:000025c0       $unwind$syncDebuggeeStatus 00000001800075c0     libMethodBind.obj
 0002:000025c0       $unwind$__scrt_dllmain_exception_filter 00000001800075c0     MSVCRT:utility.obj
 0002:000025d4       $unwind$Java_nsk_share_jvmti_DebugeeClass_resetAgentData 00000001800075d4     libMethodBind.obj
 0002:000025dc       $unwind$MA_checkStatus     00000001800075dc     libMethodBind.obj
 0002:000025f0       $unwind$Java_nsk_jvmti_unit_FollowReferences_FollowRefObjects_setTag 00000001800075f0     libMethodBind.obj
 0002:00002608       $unwind$Java_nsk_jvmti_unit_FollowReferences_FollowRefObjects_addRefToVerify 0000000180007608     libMethodBind.obj
 0002:00002624       $unwind$Agent_Initialize   0000000180007624     libMethodBind.obj
 0002:00002624       $unwind$my_findLoadedClass 0000000180007624     libMethodBind.obj
 0002:00002624       $unwind$_DllMainCRTStartup 0000000180007624     MSVCRT:dll_dllmain.obj
 0002:00002634       $unwind$Java_nsk_jvmti_unit_MethodBind_JvmtiTest_GetStackTrace 0000000180007634     libMethodBind.obj
 0002:00002634       $unwind$print_method_name  0000000180007634     libMethodBind.obj
 0002:0000263c       $unwind$debug_printf       000000018000763c     libMethodBind.obj
 0002:00002648       $unwind$testNativeMethodBind 0000000180007648     libMethodBind.obj
 0002:00002654       $unwind$Java_nsk_jvmti_unit_MethodBind_JvmtiTest_CreateRawMonitor 0000000180007654     libMethodBind.obj
 0002:00002668       $unwind$capture_previous_context 0000000180007668     MSVCRT:gs_report.obj
 0002:00002674       $unwind$__GSHandlerCheckCommon 0000000180007674     MSVCRT:gshandler.obj
 0002:00002680       $xdatasym                  0000000180007680     MSVCRT:amdsecgs.obj
 0002:00002684       $unwind$?dllmain_crt_process_attach@@YAHQEAUHINSTANCE__@@QEAX@Z 0000000180007684     MSVCRT:dll_dllmain.obj
 0002:000026c0       $unwind$?fin$0@?0??dllmain_crt_process_attach@@YAHQEAUHINSTANCE__@@QEAX@Z@4HA 00000001800076c0     MSVCRT:dll_dllmain.obj
 0002:000026c0       $unwind$?fin$0@?0??dllmain_crt_process_detach@@YAH_N@Z@4HA 00000001800076c0     MSVCRT:dll_dllmain.obj
 0002:000026c0       $unwind$?fin$1@?0??dllmain_crt_process_detach@@YAH_N@Z@4HA 00000001800076c0     MSVCRT:dll_dllmain.obj
 0002:000026c8       $unwind$?dllmain_crt_process_detach@@YAH_N@Z 00000001800076c8     MSVCRT:dll_dllmain.obj
 0002:0000271c       $unwind$?dllmain_dispatch@@YAHQEAUHINSTANCE__@@KQEAX@Z 000000018000771c     MSVCRT:dll_dllmain.obj
 0002:00002744       $unwind$?filt$0@?0??dllmain_dispatch@@YAHQEAUHINSTANCE__@@KQEAX@Z@4HA 0000000180007744     MSVCRT:dll_dllmain.obj
 0002:0000274c       $unwind$__scrt_is_nonwritable_in_current_image 000000018000774c     MSVCRT:utility.obj
 0002:0000276c       $unwind$__scrt_is_nonwritable_in_current_image$filt$0 000000018000776c     MSVCRT:utility.obj
 0002:00002774       $unwind$__scrt_fastfail    0000000180007774     MSVCRT:utility_desktop.obj
 0002:00002784       $unwind$__security_init_cookie 0000000180007784     MSVCRT:gs_support.obj
 0002:00002790       $unwind$__isa_available_init 0000000180007790     MSVCRT:cpu_disp.obj
 0002:000027a0       $xdatasym                  00000001800077a0     MSVCRT:guard_dispatch.obj
 0002:000027a8       $xdatasym                  00000001800077a8     MSVCRT:guard_xfg_dispatch.obj
 0002:000027b0       .edata                     00000001800077b0     MethodBind.exp
 0002:000027d8       rgpv                       00000001800077d8     MethodBind.exp
 0002:00002838       rgszName                   0000000180007838     MethodBind.exp
 0002:00002898       rgwOrd                     0000000180007898     MethodBind.exp
 0002:000028c8       szName                     00000001800078c8     MethodBind.exp
 0002:000028d7       $N00001                    00000001800078d7     MethodBind.exp
 0002:000028e6       $N00002                    00000001800078e6     MethodBind.exp
 0002:000028f3       $N00003                    00000001800078f3     MethodBind.exp
 0002:00002938       $N00004                    0000000180007938     MethodBind.exp
 0002:00002975       $N00005                    0000000180007975     MethodBind.exp
 0002:000029bd       $N00006                    00000001800079bd     MethodBind.exp
 0002:000029fd       $N00007                    00000001800079fd     MethodBind.exp
 0002:00002a3a       $N00008                    0000000180007a3a     MethodBind.exp
 0002:00002a74       $N00009                    0000000180007a74     MethodBind.exp
 0002:00002aab       $N00010                    0000000180007aab     MethodBind.exp
 0002:00002ade       $N00011                    0000000180007ade     MethodBind.exp
 0002:00002b15       $N00012                    0000000180007b15     MethodBind.exp
 0002:00002b4e       $N00013                    0000000180007b4e     MethodBind.exp
 0002:00002b86       $N00014                    0000000180007b86     MethodBind.exp
 0002:00002bc0       $N00015                    0000000180007bc0     MethodBind.exp
 0002:00002bf8       $N00016                    0000000180007bf8     MethodBind.exp
 0002:00002c30       $N00017                    0000000180007c30     MethodBind.exp
 0002:00002c6b       $N00018                    0000000180007c6b     MethodBind.exp
 0002:00002c99       $N00019                    0000000180007c99     MethodBind.exp
 0002:00002cca       $N00020                    0000000180007cca     MethodBind.exp
 0002:00002cf9       $N00021                    0000000180007cf9     MethodBind.exp
 0002:00002d28       $N00022                    0000000180007d28     MethodBind.exp
 0002:00002d5d       $N00023                    0000000180007d5d     MethodBind.exp
 0002:00002d6c       $N00024                    0000000180007d6c     MethodBind.exp
 0002:00003182       .idata$6                   0000000180008182     kernel32:KERNEL32.dll
 0002:000031f0       .idata$6                   00000001800081f0     vcruntime:VCRUNTIME140.dll
 0002:0000335c       .idata$6                   000000018000835c     ucrt:api-ms-win-crt-runtime-l1-1-0.dll
 0002:0000337e       .idata$6                   000000018000837e     ucrt:api-ms-win-crt-stdio-l1-1-0.dll
 0002:0000339e       .idata$6                   000000018000839e     ucrt:api-ms-win-crt-string-l1-1-0.dll
 0003:00000000       ?codeAttributeName@@3PEBDEB 0000000180009000     libMethodBind.obj
 0003:00000008       ?lineNumberAttributeName@@3PEBDEB 0000000180009008     libMethodBind.obj
 0003:00000010       ?localVarAttributeName@@3PEBDEB 0000000180009010     libMethodBind.obj
 0003:00000018       ?localVarTypeAttributeName@@3PEBDEB 0000000180009018     libMethodBind.obj
 0003:00000020       ?stackMapAttributeName@@3PEBDEB 0000000180009020     libMethodBind.obj
 0003:00000028       ?callBytes@@3PAEA          0000000180009028     libMethodBind.obj
 0003:0000002c       ?allocBytes@@3PAEA         000000018000902c     libMethodBind.obj
 0003:0001ea10       nsk_context                0000000180027a10     libMethodBind.obj
 0003:0001ea1c       redefineAttempted          0000000180027a1c     libMethodBind.obj
 0003:0001ea20       redefineSucceed            0000000180027a20     libMethodBind.obj
 0003:0001ea24       agentFailed                0000000180027a24     libMethodBind.obj
 0003:0001ea28       agentThread                0000000180027a28     libMethodBind.obj
 0003:0001ea30       context                    0000000180027a30     libMethodBind.obj
 0003:0001eae8       agentThreadProc            0000000180027ae8     libMethodBind.obj
 0003:0001eaf0       agentThreadArg             0000000180027af0     libMethodBind.obj
 0003:0001eaf8       agent_data                 0000000180027af8     libMethodBind.obj
 0003:0001eb08       jvmti_env                  0000000180027b08     libMethodBind.obj
 0003:0001eb10       jvm                        0000000180027b10     libMethodBind.obj
 0003:0001eb18       jni_env                    0000000180027b18     libMethodBind.obj
 0003:0001eb20       currentAgentStatus         0000000180027b20     libMethodBind.obj
 0003:0001eb24       ?codeAttributeIndex@@3GA   0000000180027b24     libMethodBind.obj
 0003:0001eb28       checkStatus_func           0000000180027b28     libMethodBind.obj
 0003:0001eb30       ?lineNumberAttributeIndex@@3GA 0000000180027b30     libMethodBind.obj
 0003:0001eb34       ?localVarAttributeIndex@@3GA 0000000180027b34     libMethodBind.obj
 0003:0001eb38       ?localVarTypeAttributeIndex@@3GA 0000000180027b38     libMethodBind.obj
 0003:0001eb3c       ?stackMapAttributeIndex@@3GA 0000000180027b3c     libMethodBind.obj
 0003:0001eb40       ?stackFrameOffset@@3GA     0000000180027b40     libMethodBind.obj
 0003:0001eb44       ?mode@@3HA                 0000000180027b44     libMethodBind.obj
 0003:0001eb48       ?orig@@3PEBEEB             0000000180027b48     libMethodBind.obj
 0003:0001eb50       ?gen@@3PEAEEA              0000000180027b50     libMethodBind.obj
 0003:0001eb58       ?inputPos@@3PEAEEA         0000000180027b58     libMethodBind.obj
 0003:0001eb60       ?endPos@@3PEBEEB           0000000180027b60     libMethodBind.obj
 0003:0001eb68       ?genPos@@3PEAEEA           0000000180027b68     libMethodBind.obj
 0003:0001eb70       ?markPos@@3PEAEEA          0000000180027b70     libMethodBind.obj
 0003:0001eb78       ?constantPool@@3PEAPEADEA  0000000180027b78     libMethodBind.obj
 0003:0001eb80       ?constantPoolSize@@3GA     0000000180027b80     libMethodBind.obj
 0003:0001eb84       ?constantPoolCount@@3GA    0000000180027b84     libMethodBind.obj
 0003:0001eb88       ?zeroBytes@@3PAEA          0000000180027b88     libMethodBind.obj
 0003:0001eb8c       ?codeLength@@3IA           0000000180027b8c     libMethodBind.obj
 0003:0001eb90       ?map@@3PEAIEA              0000000180027b90     libMethodBind.obj
 0003:0001eb98       ?widening@@3PEACEA         0000000180027b98     libMethodBind.obj
 0003:0001eba0       callbacks                  0000000180027ba0     libMethodBind.obj
 0003:0001ecd8       jvmti_caps                 0000000180027cd8     libMethodBind.obj
 0003:0001ecf0       GS_ExceptionRecord         0000000180027cf0     MSVCRT:gs_report.obj
 0003:0001ed90       GS_ContextRecord           0000000180027d90     MSVCRT:gs_report.obj
 0003:0001f260       ?g_tss_cv@@3U_RTL_CONDITION_VARIABLE@@A 0000000180028260     MSVCRT:thread_safe_statics.obj
 0003:0001f268       ?g_tss_event@@3PEAXEA      0000000180028268     MSVCRT:thread_safe_statics.obj
 0003:0001f270       ?g_tss_mutex@@3U_RTL_CRITICAL_SECTION@@A 0000000180028270     MSVCRT:thread_safe_statics.obj
 0003:0001f298       ?g_sleep_condition_variable_cs@@3P6AHPEAU_RTL_CONDITION_VARIABLE@@PEAU_RTL_CRITICAL_SECTION@@K@ZEA 0000000180028298     MSVCRT:thread_safe_statics.obj
 0003:0001f2a0       ?g_wake_all_condition_variable@@3P6AXPEAU_RTL_CONDITION_VARIABLE@@@ZEA 00000001800282a0     MSVCRT:thread_safe_statics.obj
 0003:0001f2ac       ?__proc_attached@@3HA      00000001800282ac     MSVCRT:dll_dllmain.obj
 0003:0001f2c0       ?is_initialized_as_dll@@3_NA 00000001800282c0     MSVCRT:utility.obj
 0003:0001f2c1       ?module_local_atexit_table_initialized@@3_NA 00000001800282c1     MSVCRT:utility.obj
 0003:0001f2c8       ?module_local_atexit_table@@3U_onexit_table_t@@A 00000001800282c8     MSVCRT:utility.obj
 0003:0001f2e0       ?module_local_at_quick_exit_table@@3U_onexit_table_t@@A 00000001800282e0     MSVCRT:utility.obj
